:1000000009C016C015C014C013C012C011C010C062
:1000100029C00EC011241FBECFE9CDBF10E0A0E65D
:10002000B0E001C01D92A239B107E1F749D008C183
:10003000E7CF89BD86BF0895369A3699FECF95B130
:10004000981760F4809160008F5F893018F4809376
:10005000600006C01092600081E008951092600078
:1000600080E008951F920F920FB60F9211242F93E4
:100070003F938F939F93809167008F3F19F08F5F1D
:100080008093670080916700803F88F02091640032
:1000900030E08091610090E001972817390739F42A
:1000A00089B58D3820F089B5815089BD86BF9F9173
:1000B0008F913F912F910F900FBE0F901F90189529
:1000C00089E188BB82E087BB81E687B9A29A86EC8A
:1000D00086B9479A80916100E82FF0E0E859FF4F18
:1000E0009FEF90838F5F8093610085B7877E85BF88
:1000F000F894A89581B5886181BD85E481BD789427
:10010000E0916400F0E0E859FF4F8081893010F001
:1001100083E201C081E28FBD81E083BFE091640092
:10012000F0E0E859FF4F808189BD86BFC7E082E8D3
:1001300083DF882309F47CC080916400811138C07A
:1001400086B78830A8F588E777DF8823E1F38BE06E
:1001500014C02FE739EA43E0215030404040E1F736
:1001600000C00000C9BDC6BF9FEF22E537E0915037
:1001700020403040E1F700C00000815019BC16BE9D
:100180008111E7CFF894A89584B7877F84BF81B5A4
:10019000886181BD11BC789485B7877E806185BFF9
:1001A00085B7806285BF889585B78F7D85BF37C04D
:1001B00096B784E016C019BC16BE4FE729EA33E0B3
:1001C000415020403040E1F700C0000099BD96BF8B
:1001D0004FEF22E537E0415020403040E1F700C0CA
:1001E0000000815041F786B7803128F086B78695A8
:1001F00089BD86BF02C0C9BDC6BF80916400882387
:1002000071F096B7E0916400F0E0E859FF4F80810B
:10021000981728F4809164008150809364004FEF18
:1002200081EF9BE2415080409040E1F700C0000028
:1002300085B7806285BF889585B78F7D85BF77CF6D
:04024000F894FFCF60
:00000001FF
